:020000040000FA
:060000008B018A01332888
:080008008C102008031D1028D4
:100010000608C039083886001F150130A1002D28B8
:10002000013A031D1C286220023E9F1DA2009F1959
:10003000A30008309F062D288611220820060319E8
:10004000061623082006031986160608F839210427
:1000500086000130A10DA119A100A00ACA30200616
:100060000319A00109008601850183161F30850050
:10007000860160308F009001803081008C018D01FD
:10008000C0309F00831241309F008C018D01831688
:10009000453092008C14831204309200A001A1011B
:1000A000A201A3018B170B1754289E0183169E01F2
:1000B000831262200000031383169E0A8312031921
:1000C0009E0A59286E3083161E078312A400003042
:1000D0000318013E1E078A00240882000034013400
:1000E00002340334043405340634073408340B3442
:1000F0000F34133416341A341D341F34223424348C
:10010000263429342B342D342E34303432343334E5
:1001100035343634383439343B343C343D343E3471
:100120004034413442344334443445344634473413
:10013000483449344A344B344C344C344D344E34C6
:100140004F34503450345134523453345334543483
:100150005534553456345734573458345934593447
:100160005A345A345B345C345C345D345D345E3410
:100170005E345F345F3460346034613461346234DF
:1001800062346334633464346434653465346634AF
:100190006634663467346734683468346934693483
:1001A00069346A346A346B346B346B346C346C3459
:1001B0006C346D346D346E346E346E346F346F3431
:1001C0006F3470347034703471347134713472340B
:1001D00072347234733473347334743474347434E6
:1001E00075347534753475347634763476347734C2
:1001F00077347734773478347834783479347934A0
:10020000793479347A347A347A347A347B347B347E
:100210007B347B347C347C347C347D347D347D345D
:100220007D347D347E347E347E347E347F347F343E
:100230007F347F348034803480348034813481341E
:100240008134813481348234823482348234823401
:1002500083348334833483348434843484348434E2
:1002600084348534853485348534853486348634C5
:1002700086348634863487348734873487348734A9
:10028000873488348834883488348834893489348D
:100290008934893489348A348A348A348A348A3471
:1002A0008A348B348B348B348B348B348B348C3456
:1002B0008C348C348C348C348C348D348D348D343B
:1002C0008D348D348D348E348E348E348E348E3421
:1002D0008E348F348F348F348F348F348F348F3407
:1002E00090349034903490349034903491349134EC
:1002F00091349134913491349134923492349234D3
:1003000092349234923492349334933493349334B9
:1003100093349334933494349434943494349434A0
:100320009434943495349534953495349534953487
:10033000953495349634963496349634963496346F
:100340009634963497349734973497349734973457
:10035000973497349834983498349834983498343F
:100360009834983499349934993499349934993427
:10037000993499349A349A349A349A349A349A340F
:100380009A349A349B349B349B349B349B349B34F7
:100390009B349B349B349C349C349C349C349C34E0
:1003A0009C349C349C349C349D349D349D349D34C9
:1003B0009D349D349D349D349D349E349E349E34B2
:1003C0009E349E349E349E349E349E349E349F349C
:1003D0009F349F349F349F349F349F349F349F3485
:1003E000A034A034A034A034A034A034A034A0346D
:1003F000A034A034A134A134A134A134A134A13457
:10040000A134A134A134A134A234A234A234A23440
:10041000A234A234A234A234A234A234A234A3342B
:10042000A334A334A334A334A334A334A334A33414
:10043000A334A434A434A434A434A434A434A434FD
:10044000A434A434A434A434A534A534A534A534E8
:10045000A534A534A534A534A534A534A534A534D4
:10046000A634A634A634A634A634A634A634A634BC
:10047000A634A634A634A734A734A734A734A734A7
:10048000A734A734A734A734A734A734A734A83493
:10049000A834A834A834A834A834A834A834A8347C
:1004A000A834A834A834A934A934A934A934A93467
:1004B000A934A934A934A934A934A934A934A93454
:1004C000AA34AA34AA34AA34AA34AA34AA34AA343C
:1004D000AA34AA34AA34AA34AB34AB34AB34AB3428
:1004E000AB34AB34AB34AB34AB34AB34AB34AB3414
:1004F000AB34AC34AC34AC34AC34AC34AC34AC34FD
:10050000AC34AC34AC34AC34AC34AC34AC34AD34EA
:10051000AD34AD34AD34AD34AD34AD34AD34AD34D3
:10052000AD34AD34AD34AD34AD34AE34AE34AE34C0
:10053000AE34AE34AE34AE34AE34AE34AE34AE34AB
:10054000AE34AE34AE34AF34AF34AF34AF34AF3496
:10055000AF34AF34AF34AF34AF34AF34AF34AF3483
:10056000AF34B034B034B034B034B034B034B0346C
:10057000B034B034B034B034B034B034B034B0345B
:10058000B134B134B134B134B134B134B134B13443
:10059000B134B134B134B134B134B134B134B23432
:1005A000B234B234B234B234B234B234B234B2341B
:1005B000B234B234B234B234B234B234B234B3340A
:1005C000B334B334B334B334B334B334B334B334F3
:1005D000B334B334B334B334B334B334B334B434E2
:1005E000B434B434B434B434B434B434B434B434CB
:1005F000B434B434B434B434B434B434B434B534BA
:10060000B534B534B534B534B534B534B534B534A2
:10061000B534B534B534B534B534B534B534B53492
:10062000B634B634B634B634B634B634B634B6347A
:10063000B634B634B634B634B634B634B634B6346A
:10064000B634B734B734B734B734B734B734B73453
:10065000B734B734B734B734B734B734B734B73442
:10066000B734B734B734B834B834B834B834B8342D
:10067000B834B834B834B834B834B834B834B8341A
:10068000B834B834B834B834B834B934B934B93407
:10069000B934B934B934B934B934B934B934B934F2
:1006A000B934B934B934B934B934B934B934B934E2
:1006B000BA34BA34BA34BA34BA34BA34BA34BA34CA
:1006C000BA34BA34BA34BA34BA34BA34BA34BA34BA
:1006D000BA34BA34BA34BB34BB34BB34BB34BB34A5
:1006E000BB34BB34BB34BB34BB34BB34BB34BB3492
:1006F000BB34BB34BB34BB34BB34BB34BB34BC3481
:10070000BC34BC34BC34BC34BC34BC34BC34BC3469
:10071000BC34BC34BC34BC34BC34BC34BC34BC3459
:10072000BC34BC34BC34BD34BD34BD34BD34BD3444
:10073000BD34BD34BD34BD34BD34BD34BD34BD3431
:10074000BD34BD34BD34BD34BD34BD34BD34BE3420
:10075000BE34BE34BE34BE34BE34BE34BE34BE3409
:10076000BE34BE34BE34BE34BE34BE34BE34BE34F9
:10077000BE34BE34BE34BE34BE34BF34BF34BF34E6
:10078000BF34BF34BF34BF34BF34BF34BF34BF34D1
:10079000BF34BF34BF34BF34BF34BF34BF34BF34C1
:1007A000BF34BF34C034C034C034C034C034C034AB
:1007B000C034C034C034C034C034C034C034C03499
:1007C000C034C034C034C034C034C034C034C03489
:1007D000C134C134C134C134C134C134C134C13471
:1007E000C134C134C134C134C134C134C134C13461
:1007F000C134C134C134C134C134C134C134C23450
:10080000C234C234C234C234C234C234C234C23438
:10081000C234C234C234C234C234C234C234C23428
:10082000C234C234C234C234C234C234C234C33417
:10083000C334C334C334C334C334C334C334C33400
:10084000C334C334C334C334C334C334C334C334F0
:10085000C334C334C334C334C334C334C334C434DF
:10086000C434C434C434C434C434C434C434C434C8
:10087000C434C434C434C434C434C434C434C434B8
:10088000C434C434C434C434C434C434C434C534A7
:10089000C534C534C534C534C534C534C534C53490
:1008A000C534C534C534C534C534C534C534C53480
:1008B000C534C534C534C534C534C534C534C53470
:1008C000C534C634C634C634C634C634C634C63459
:0C08D000C634C634C634C634C634C63440
:084000000000010000000100B6
:02400E00503F21
:00000001FF
